:03000000021039B2
:03000B000200A24E
:03002B000202CB03
:03005B0002041587
:030073000203EF96
:1000800002030406080C10182030406080040608A3
:100090000C10182030406080A0C005050D0502033B
:1000A0000302C2AFC0D0C0E020622C20680241B77A
:1000B0003066024177302F02E4730563C3740595FF
:1000C0002540F5956340F12069EE758A78E5257045
:1000D00003758A000202C485258AC262E525F47090
:1000E00002213E206802212B758B00D0E0D0D0D2B7
:1000F00097D295D293D2AF32D297D295D293740140
:10010000D5E0FDE53C1420E21520E10D207D02D272
:1001100094307D02D29602013BD29202013B207DB7
:1001200002D296307D02D29402013B758B00D0E062
:10013000D0D0D297D295D293D2AF32758B00D0E087
:10014000D0D0D2AF3241B7E525600A207D02C297F8
:10015000307D02C295D29341B7E5256002C293205B
:100160007D02D295307D02D29741B7E525600A2005
:100170007D02C295307D02C297207D02D297307DEC
:1001800002D29541B7207D02C296307D02C29420F2
:100190007D02C294307D02C2967419D5E0FDE5253A
:1001A000600A207D02C297307D02C295D29341B78A
:1001B000207D02C296307D02C294C2927419D5E0AD
:1001C000FDE525600A207D02C297307D02C295D2EE
:1001D0009341B7C292207D02C296307D02C29474D0
:1001E00019D5E0FDE5256002C293207D02D295304D
:1001F0007D02D29741B7C292207D02C294307D0227
:10020000C2967419D5E0FDE5256002C293207D02F7
:10021000D295307D02D29741B7207D02C294307DC5
:1002200002C296C2927419D5E0FDE525600A207DD0
:1002300002C295307D02C297207D02D297307D02A6
:10024000D29541B7207D02C294307D02C296207DB6
:1002500002C296307D02C2947419D5E0FDE5256096
:100260000A207D02C295307D02C297207D02D2977E
:10027000307D02D29541B730723DE53C20E21A2034
:10028000E129207D02C296307D02C294207D02C207
:1002900094307D02C2960202B720E1E6207D02C2C0
:1002A00096307D02C294C2920202B7C292207D02B1
:1002B000C294307D02C296E525F4F58A758B0075EF
:1002C0006300D262D0E0D0D0D2AF32C2AFC2AD5361
:1002D000E6EFC0D0C0E0D2D3D2AFC2CEE5296007EE
:1002E0002074461529612978007900E580307E0167
:1002F000F430E50278FF53DACF207E0343DA203072
:100300007E0343DA10C2D8C271E580307E01F4303A
:10031000E50279FFC3E89970CE3061037529182092
:1003200074037529188859D270E52A6004152A616A
:100330003920740543DA01C2D82070026194A859AB
:10034000206102C270207431C3E894F0400374F05D
:10035000F8E8C4540F28F87984B703026179C3130D
:10036000C3138721200802C313200A06C3C898F8C4
:10037000617928F8500374FFF8C3E895625003E5EB
:1003800062F8882230690AC3E522955E4003855EE3
:1003900022852224A824C3E524955E4002A85E8815
:1003A00025C3E52594404002D26420CF0CD0E0D094
:1003B000D0C2D343E610D2AD32C2CF7801E5296076
:1003C000053074021529C3E55994014005755C0098
:1003D00061E3755D00756400E55C2401F55C500324
:1003E000755CFFD0E0D0D0C2D343E610D2AD32C0AE
:1003F000D0C0E0C2AF53917F53E67FC260759100D9
:10040000C3E49550F594E49551F595759104D0E0C9
:10041000D0D0D2AF32C2AF53E6EFC2ADC0D0C0E051
:10042000C0F0D2D3D2AFA8FBA9FCC2D830710281F0
:100430007C53DACF207E0343DA10307E0343DA2088
:10044000D271E580307E01F420E50281538826894F
:1004500027C1B853DACF207E0343DA20307E03432E
:10046000DA10C2D8C271307402C1A47800E58030BD
:0F0470007E01F430E502C1A48859C18B53DACF65
:10047F00207E0343DA20307E0343DA10C2712061FD
:10048F0002A14C53DACF207E0343DA10307E0343B0
:10049F00DA20C2D8D27188548955C3E89552F8E949
:1004AF009553F9E4FB7E027A00C3E8948CE994003B
:1004BF005005755800A13CC3E894C8E99400500852
:1004CF00E4D2E4FB7A0AA119C3E89468E9940150D5
:1004DF0008E4D2E3FB7A0FA119C3E894D0E99402A0
:1004EF005008E4D2E2FB7A1EA119C3E894A0E99464
:1004FF00055008E4D2E1FB7A3CA119C3E89498E9CE
:10050F0094085008E4D2E0FB7A787E00C3E8955651
:10051F00FCE99557FD30E708ECF42401FCEDF4FD00
:10052F00755800C3EC9AED9E500375580188568993
:10053F0057A854A955885289537802C18BC3E8959F
:10054F0026F8E99527F9307C02C16F307B02C16F25
:10055F00307A02C168207502A16FE9FDE8FCA18E17
:10056F00E9C313F9E813F8307902C168E9C313F945
:10057F00E813F8307802C168E9C313FDE813FC20D3
:10058F006126C3EC941CED94024002A1A5ED7018F6
:10059F00C3EC94C850120528C3E528940A5002C131
:1005AF00A4755900D270C1A4E52860021528740003
:1005BF00207F0B7888E67896B40302789EE624FABB
:1005CF00FEE43400FFC3EC9EFCED9FFD920878889B
:1005DF00E6B40327A2085009207D20C2AFD27DA127
:1005EF00F7307D17C2AFC27DD297D295D293C29604
:1005FF00C294C292206902D26BD2AFA2085017E602
:10060F00B4030DECF42401FCEDF43400FD020625D7
:10061F0078007900C16F7888E6B40315EC33FCEDF0
:10062F0033FDC3EC940AFCED9400FD50047C007D77
:10063F0000C3EC94FFED9400400678FF7900C16F82
:10064F00EC856FF0A4C5F0A2F733F87900400302F0
:10065F00068B78FF790002068BE9C313F9E813F8CC
:10066F00307C0EE9600278FFC3E81338F8E43400F9
:10067F00F9C3E894FFE99400400278FF8859D270DB
:10068F00206102C1A4741FF4552F4BF52FC274E4DF
:10069F002B7002D27475291830740375290A3061D2
:1006AF0002C1B820740353DAFE752A06307403753D
:1006BF002A0AD0F0D0E0D0D0C2D3D2AD43E6103268
:1006CF0079010206ED79030206ED790A0206ED794A
:1006DF001E0206ED79640206ED79C80206ED781761
:1006EF00E4D5E0FDD8FAD9F6227A147B7802071404
:1006FF007A107B8C0207147A0D7BB40207147A0BE5
:10070F007BC8020714AC257525017902B27DE4C2BE
:10071F0092D5E0FDE5256002C293D5E0FDD293D5D9
:10072F00E0FDD292D5E0FDE525600A207D02C2975B
:10073F00307D02C295E570D5E0FD207D02D2973065
:10074F007D02D2957496D5E0FDD9C1EAF8D5E0FDCA
:10075F00D8FBDBB1C2928C2522C37C007D0075F0E3
:10076F000005F0EA33FAEB33FB50F6EB13FBEA1319
:10077F00FAC3E9FFE8FEE89AF8E99BF95004EFF9AC
:10078F00EEF8B3EC33FCED33FDD5F0DFEDF9ECF81B
:10079F0022E889F08A20D2D4F8A9F07B0030F70B39
:1007AF007BFFF42401F8E9F43400F9E88520F0A484
:1007BF00ADF0F8E98520F0A4AFF0FEED2EF974004E
:1007CF003FFA7C04C3EA13FAE913F9E813F8DCF4EF
:1007DF008BF030F70AE8F42401F8E9F43400F9E873
:1007EF0089F0C2D4F8A9F02222E547603BC3E53B6C
:1007FF0013F9E53A13F8C3E53E98F8E53F99F95038
:10080F000CC3E89480E994FF4016020833C3E894C0
:10081F007FE994005003020833787F790002083390
:10082F00788079FF8843894422E5476058E543255E
:10083F0040F8E5443541F9854420E4300701F435AB
:10084F0042FA30E709C3EA94F04015020875C3EA8B
:10085F00940F500302087578FF79FF7A0F0208751D
:0F086F00780079007AF0C3E524955E5006E52401
:10087E006009018EE54420E70D018EE54430E70660
:10088E00884089418A4222E54770030208F978A11F
:10089E00E6FAC3E54333F8E54433F91207A0E9302D
:1008AE00E70BC3E89480E994FF401301D0C3E894AA
:1008BE007FE99400500201D0787F790001D07880D2
:1008CE0079FFE820E715C3E52398F84009C3E894BB
:1008DE000140030208F778010208F7E8F424012525
:1008EE0023F840030208F778FF884522E547700396
:1008FE0002095C78A2E6FAA841A9421207A0E930E3
:10090E00E70CC3E89401E994FF4016020933C3E8EB
:10091E0094FFE99400500302093378FF790002092D
:10092E0033780179FFE920E715C3E54598F84009CA
:10093E00C3E89401400302095A780002095AE8F408
:10094E0024012545F8400302095A78FF88242278AD
:10095E00FFC264E52D5406702FD264C3E53B940AA2
:10096E004009C3E52594405002C264E53B6019740A
:10097E00FF853BF0848537F0A4F8C5F0600278FF60
:10098E00C3E895615002A861886022020A36788316
:10099E00E6F520120E5F75E8901206CF75E890E529
:1009AE00E820ECFBA8BDA9BE120EF5756B55756C53
:1009BE0000C3740013FD745513FC74552CFC7400A5
:1009CE003DFDECFAEDFBC3E89AE99B4014E56B2480
:1009DE0055F56BE56C3400F56CEA2CFAEB3DFB80BB
:1009EE00E5AE6BAF6CC3E56C13F9E56B13F8C3E9B9
:1009FE0013F9E813F8E56B28F569E56C39F56A7AB1
:100A0E0003C3E913F9E813F8DAF7AA201A70097587
:100A1E006B00756C00020A361AEA6008EE28FEEFCB
:100A2E0039FFDAF88E6B8F6C2275E890227883E6A8
:100A3E00FFE5E820ECF7A8BDA9BE056DC3E56D94F2
:100A4E00084052756D00E9FA79A0E76044EA700734
:100A5E00E56E601B020A71C3E8956E6010E56E507C
:100A6E0006600C14020A7D0460F9020A7DE56EF53B
:100A7E006EC3946D401B755EC0C394044013755EC7
:100A8E0080C39404400B755E40C394044003755EAE
:100A9E000075BB0822E55EF46002055EE56DB407E5
:100AAE000375BB1022743279A387F0A4C5F0A2F7A8
:100ABE0033F8C3E8955E4002A85E88228824882514
:100ACE00886122753A00753B7F2275C820A8CCA993
:100ADE00CD75C824AA38AB3988388939C3E89AF855
:100AEE00E99BF9AA3AAB3BAC3AAD3B7E047F02C31D
:100AFE00EB940440021E1FC3EB940840021E1FC35A
:100B0E00ED13FDEC13FCDEF7C3EA9CFAEB9DFBEF55
:100B1E006009C3E913F9E813F8DFF7EA28FAEB39AD
:100B2E00FB8A3A8B3B400122753AFF753BFF223020
:100B3E006002613D854C50854D51D26043E6802266
:100B4E007892E6FFC3E535948240010FC3E53594F4
:100B5E00A040010FC3EF940640027F057E021E30B7
:100B6E0072010EC3E53B940350060E0E3072010E59
:100B7E00C3E53B940250060E0E3072010EA93BA83F
:100B8E003A7A04C3E913F9E813F8DAF7C3E89EF8E2
:100B9E00E99400F94009C3E89402E99400500478FE
:100BAE0002E4F9E9FBE8FAC3E913FDE813FC884C0B
:100BBE00894DC3EF94036037EF20E00DE82CF8E980
:100BCE003DF9ECFAEDFB020BEAE828F8E939F9C336
:100BDE00E89402F8E99400F97A02E4FBC3EF940377
:100BEE00400D8A4E8B4F884889498C4A8D4B2288FE
:100BFE004E894F8A488B498C4A8D4B223060028138
:100C0E000AD26043E680E52D54066027A83AA93B38
:100C1E00E53494085006E820E002A94D759100C312
:100C2E00E498F594E499F595759104D26053917F0B
:100C3E0043E68022D265753D00752000020C55D228
:100C4E0065753D00752040E52D54066002C265D2E3
:100C5E00AF206005E53D60012278017A02C3E53BD5
:0F0C6E00940540027802C3E53B940A40027803E4
:100C7D00C3E53B940F40027A03306904781E7A0174
:100C8D00206007E53D6003D2AF22D2AF0000C2AFB6
:100C9D00C3E53BFB940F40027B0FEB043073012344
:100CAD0020620123F93069027982E58BC39940D026
:100CBD00053DEAFBE59B5440B52004DBF781F020B0
:100CCD0065028155C265759100AE3AAF3BC3E49E96
:100CDD00F594E49FF595759104D26053917F43E6A9
:100CED008081553065028155D896D2AF2230690B7F
:100CFD000534206016753400020D1820600D206536
:100D0D000A206B071581158102150922A84EA94FDE
:100D1D0075910053917FC3E498F594E499F5957519
:100D2D009104854850854951D26043E68022780070
:100D3D003064053065027801E53575F007A4F9E5F5
:100D4D00F028F5F0E9A2F013A2F113A2F213F53594
:100D5D00C394785003753578C3E53595364008D280
:100D6D0066D297D295D293306002A174854A508590
:100D7D004B51D26043E68022C2AFC296C294C2925A
:100D8D0030720B9002197419D5E0FD020D9B207D78
:100D9D0002D296307D02D294759F13753C02020EDD
:100DAD00DAC2AF207D02D295307D02D29730721714
:100DBD009001F6C292207D02C294307D02C29674DB
:100DCD0019D5E0FD020DD7900159306206E5256079
:100DDD0002C293207D03759F10307D03759F1175A1
:100DED003C03020EDAC2AFC296C294C29230720BAD
:100DFD009001D37419D5E0FD020E08207D02D29426
:100E0D00307D02D296207D03759F11307D03759F35
:100E1D0010753C04020EDAC2AFD2933072179001F6
:100E2D00B0207D02C296307D02C294C2927419D553
:100E3D00E0FD020E4590014730620EE525600A2067
:100E4D007D02C297307D02C295759F13753C0502D8
:100E5D000EDAC2AFC296C294C29230720B90018567
:100E6D007419D5E0FD020E75D292207D03759F1089
:100E7D00307D03759F11753C06020EDAC2AF207DE1
:100E8D0002D297307D02D29530721F900244207DA0
:100E9D0002C296307D02C294207D02C294307D0242
:100EAD00C2967419D5E0FD020EBA90016B30620E38
:100EBD00E525600A207D02C295307D02C297207D16
:100ECD0003759F11307D03759F10753C01306B13B9
:100EDD00120EF57419D5E0FD7401D5E0FDD296D250
:100EED0094D292C266D2AF22900145D297D295D2BA
:100EFD0093C296C294C292C26222788076FF08761F
:100F0D00FF0876FF0876FF08760308760408760A50
:100F1D00087601087601087601788C76010876FF4F
:100F2D000876FF0876FF0876FF0876FF0876030837
:100F3D0076FF0876FF0876FF0876250876D00876C6
:100F4D00FA0876FA0876040876FF08760108760026
:100F5D0008767A0876FF087601227887E6FFC27256
:100F6D007888E6C394036008C27DE630E102D27D45
:100F7D00C27E7889E630E102D27EC3EF940260082A
:100F8D00758E01D273020F9A758E00C2732278800E
:100F9D00E6149000809378A1F67881E61490008095
:100FAD009378A2F6D1F5227886E61490008D937889
:100FBD00A3F6D1F52222789CE67536FF75370CB471
:100FCD0002067536A075370AB40306753682753775
:100FDD000522227896E6FA7897E6FB307F047A00B0
:100FED007BFFC3EB9AFCC3948250027C82756F0029
:100FFD00056FEC856FF0A4C3E5F0948040F222D22A
:10100D007F120FE01206DE7A007B007C101206D4F0
:10101D00E5592AFA74003BFBDCF37C04C3EB13FBAC
:10102D00EA13FADCF7FEC27F120FE022E5EF20E6AD
:10103D00037520000520903FFFE520146006901DEC
:10104D00FF1460009304600375EF12C2D353D9BF30
:10105D007581C043FF801206CF75EF0243B203E5E1
:0E106D00B3240420E702F5B3120EF57580FFE0
:10107B0075A40075F1B275D4DF7590A975A5FC75D3
:10108B00F2FE75D50175A60175E241120F07121517
:10109B003B78988670C2AF1206E81206F81206DE8D
:1010AB001206FF1206DE1207061206DE12164F128A
:1010BB0006E81206E81206E3C2AFE4F8F6D8FD78AC
:1010CB00C879C8308507D9FBD8F7021C00120F0767
:1010DB0012153B120F67120F9B120FB4120FC21295
:1010EB000FC3120FDF120FE078988670120EF57592
:1010FB00885075891275C82475910475D84075A8E8
:10110B002275B80275E690759B80759D0075D10EA2
:10111B0075BC5875BB0875BA1175E8801206CFD22D
:10112B00AF12099943DA01C2D8C2711206E87530C1
:10113B0001D2617B037A0CE55870067A0CDB020155
:10114B00C31206DE20700201C3C270E559C39402BC
:10115B0040E3E52F541F855B5AF55BB55AD7DAD7B9
:10116B00C26153DACF207E0343DA20307E0343DAA9
:10117B0010C2D8C271C2757528001206E33074090B
:10118B00C3E528940A4002D2751206D47802307453
:10119B00027800C3E5599840F0C2AF1206F8120668
:1011AB00F81206F8D2AF1206E87546007888E6B456
:1011BB00030241981206D4788CE6C39401500302C3
:1011CB001298E530C394015003021298207435C372
:1011DB00E55994FF5003021298C2AF12070DD2AF1C
:1011EB001206E3C3E559940150EFC2AF1206F81291
:1011FB0006D91206F8D2AF1206E3C3E55994FF40A5
:10120B00E90216D47F05D27F120FE01206E3C2AFBC
:10121B00C27F120FE0AE59C3E559947FD2AF40772E
:10122B001206CFC2AF12070DD2AFDFDA110CC3EE2D
:10123B0094057897F61206E812157D1216577F0A59
:10124B00D27F120FE01206E3C2AFC27F120FE0AEE5
:10125B0059C3E559947FD2AF50E41206CFC2AF12F7
:10126B0006F81206D91206F8D2AFDFD4110CEE2411
:10127B00057896F61206E812157D1216861206E30D
:10128B00120FE0C3E55994FF40F30216D4C3E5599E
:10129B00954640038559461206E378017988E7B4F1
:1012AB0003027805C3E55998400221B7C2AF120774
:1012BB000D12070D12070DD2AF1206E8753000E4C0
:1012CB00F531F5320531E531F470390532789AE6AE
:1012DB007819146012783214600D787D14600878D8
:1012EB00FA146003753200C3E53298401715327556
:1012FB0031B478998670C2AF12070DD2AF78988649
:10130B00701206E31206D9E529700530740201C389
:10131B0078012074027806C3E5599840A77888E6CF
:10132B00C3940360031206E3E529700201C3C2AF45
:10133B00120EF5E4F522F523F524F525D2AF7885C9
:10134B008662F53EF53FF540F541F542F56DF54703
:10135B00F52CF52DF535120AD1756D0875BB1012EC
:10136B0006CF120A37E5E820ECFBA8BDA9BEE97051
:10137B0001F8886E120A3B756D0875BB107887E60D
:10138B00FE7602120F677887EEF6C2AF755EFF121C
:10139B000AB385225E85225F852260D2AF7522015A
:1013AB00752401752501855D64756501D268D26967
:1013BB00753400120E5F120E89120AD1120AD8125E
:1013CB000B4E0213DC120EF5120F67756D0075BB19
:1013DB0008120C4D120CFA120D191207F7120D3BD5
:1013EB00120D85120AD8120B3D120B4E120C0A125B
:1013FB000C42120CFA120D191207F812095D120D9C
:10140B003B120DAE120AD8120B3D120B4E120C0AE8
:10141B00120C4D120CFA120D19120838120D3B1248
:10142B000DF2120AD8120B3D120B4E120C0A120CB3
:10143B0042120CFA120D19120895120D3B120E24C2
:10144B00120AD8120B3D120B4E120C0A120C4D1233
:10145B000CFA120D191208FA120D3B120E5F120A3A
:0D146B00D8120B3D120B4E120C0A120C424F
:10147800120A37120CFA120D19120A3B120D3B12FE
:101488000E89120AD8120B3D120B4E120C0A306943
:1014980035206B3285615E85615F855D64756501A8
:1014A80079327A0AC3E53499400FC269D26A8A331D
:1014B800755EFF755FFF0214CEC3E55994014003C2
:1014C8000213DC021509306A1B206B18E53314700F
:1014D80004C26A61D0F533C3E5599401400302138D
:1014E800DC021509C3E55C94825016307404E529C2
:1014F800600FC3E53B78F0306B027860985002616A
:10150800DCC2AF120EF57887E6FE7602120F677816
:1015180087EEF6E4F522F523F524F525F562C26891
:10152800D2AF1206CF120EF5307406E5297002010B
:10153800C341CA901A0D78201215BFE520B45A0C81
:10154800A31215BFE520B4A50302155D120F0712FB
:10155800157D02157C901A0378807B0A1215BFA3AB
:1015680008DBF9901A0F788C7B151215BFA308DBDE
:10157800F9901A2422C2AF1215FE1215D8901A003B
:10158800740D1215C4A374021215C4A37413121592
:10159800C4901A0378807B0A1215C3A308DBF9905C
:1015A8001A0F788C7B151215C3A308DBF9121611D4
:1015B8001215EF901A2422E493F622E6438F015382
:1015C8008FFD75EF0275B7A575B7F1F0538FFE2241
:1015D800438F02438F0175EF0275B7A575B7F19078
:1015E8001A0DF0538FFC22901A0D745AB1C4901A38
:1015F8000E74A5B1C4227A3079D07820901A40B1FF
:10160800BFE520F709A3DAF7227A3079D0901A409B
:10161800E7B1C409A3DAF922AB71A872BB01027958
:1016280084BB02027985BB03027986BB04027992E6
:10163800BB05027987BB0602799CBB07027988BB88
:1016480008027989E8F7227C051206E8DCFB22C249
:10165800AF1206F81206FF12070612070D1206D976
:101668001206F81206FF12070612070D1206D91203
:1016780006F81206FF12070612070DD2AF22C2AFF4
:1016880012070D1207061206FF1206F81206D912E3
:10169800070D1207061206FF1206F81206D91207DE
:1016A8000D1207061206FF1206F8D2AF22AE71AF6E
:1016B80072C2AF1206F81206F81206F81206D9DE40
:1016C800F212070D1206D9DFF8D2AF22D157D14F47
:1016D800D14F757101757201757300D1B57C05AD77
:1016E800591206E8C3ED955970F5C3E559940140C0
:1016F8000AC3E55994FF4032021710D120B17DD1B9
:1017080057C2AF75EF12D14FDCD50573C3E573949B
:1017180003500280C6D14F0572E5711490009A9368
:10172800F808C3E57298500280AED14FD14F0571C9
:10173800C3E57194095002809C120F07B17DC2AFB6
:0517480075EF12D14F06
:101A00000D0213FFFFFFFF03040A0101015AA501A4
:101A1000FFFFFFFFFF03FFFFFF25D0FAFA04FF01DE
:051A2000007AFF01FF48
:101A4000235475726E696779313841232020202034
:101A500023424C48454C4923463333302320202031
:101A60002020202020202020202020202020202076
:101C0000C2AFC2D353D9BF7581C043B20343FF8073
:101C1000752438752503B1BF75EF0275E24043F1B5
:101C20002053A4DFD285780379E67C1075220075F5
:101C30002300901DCC7B0675249875250130850204
:101C4000813D208508D8FBD9F9DCF781AD308508C6
:101C5000D8FBD9F9DCF781ADB17FE493A3C39A60D7
:101C6000028126DBDDB171600281267B08E493FAF4
:101C7000A3B152DBF87A30B152752200752300B15E
:101C800071EAFCEBFDC3ED94FE400EB1718A278B27
:101C900028ED30E0048A828B83B1717AC270D8C398
:101CA000ED94FE601050CEBD0022EC600675200061
:101CB0000200008100A827A9280809D804D90281B8
:101CC000C9B175EA89AAF281BB0D8199C3ED94036C
:101CD0005049EDA2E092007AC5C3E5829400E58305
:101CE000941C5093200010438F02438F0175B7A5B9
:101CF00075B7F1F030001FA827A9280809438F0104
:101D0000538FFDD804D902A11689AAE275B7A5752B
:101D1000B7F1F0A3A103538FFC81757AC1BD030C09
:101D2000E493A3FAB136DCF8B12E81758177AA224B
:101D3000AB23B152EBFAEA6222752608C3E52313FE
:101D4000F523E52213F52250066323A0632201D573
:101D500026EAB1BFB1BF75260AEAF4200102D28596
:101D6000300102C285B1BFC3134002C201D526EBC8
:101D700022B175EAFB208502A175308502A17A7532
:101D80002608AE24AF25C3EF13FFEE13FEB1C3B197
:101D9000BFC3EA133085024480FA30E703632201AF
:101DA000C3E52313F523E52213F52250066323A090
:101DB000632201D526D9E52265236523F52222AECB
:101DC00024AF250E0FDEFEDFFCD20122424C486517
:0A1DD0006C6934373132F33006013C
:00000001FF
